** EXPERIMENTAL (HLL) ** Open Watcom Linker Version 1.6beta1 Limited Availability
Portions Copyright (c) 1985-2002 Sybase, Inc. All Rights Reserved.
Created on:       13/11/17 16:25:07
Warning! W1121: file U:/tmp\ldconv_socketmodule_obj_19ea52885a3a128c58.obj(U:\DEV\python-2.7.5\Modules\socketmodule.c): '_init_socket' has already been exported
Executable Image: build/lib.os2knix-2.7/_socket.pyd
creating an OS/2 EMX dynamic link library


                        +------------+
                        |   Groups   |
                        +------------+

Group                           Address              Size
=====                           =======              ====

CGROUP                          0001:00000000        000096b0
DGROUP                          0002:00000000        00003e80



                        +--------------+
                        |   Segments   |
                        +--------------+

Segment                Class          Group          Address         Size
=======                =====          =====          =======         ====

TEXT32                 CODE           CGROUP         0001:00000000   000096b0
________TEXT           CODE           CGROUP         0001:000096b0   00000000
DATA32                 DATA           DGROUP         0002:00000000   00003cc0
SET1__os2dll           DATA           DGROUP         0002:00003cc0   00000004
SET2__os2dll           DATA           DGROUP         0002:00003cc4   00000000
SET3__os2dll           DATA           DGROUP         0002:00003cc4   00000004
SET1___CTOR_LIST__     DATA           DGROUP         0002:00003cc8   00000004
SET2___CTOR_LIST__     DATA           DGROUP         0002:00003ccc   00000000
SET3___CTOR_LIST__     DATA           DGROUP         0002:00003ccc   00000004
SET1___DTOR_LIST__     DATA           DGROUP         0002:00003cd0   00000004
SET2___DTOR_LIST__     DATA           DGROUP         0002:00003cd4   00000000
SET3___DTOR_LIST__     DATA           DGROUP         0002:00003cd4   00000004
SET1___crtinit1__      DATA           DGROUP         0002:00003cd8   00000004
SET2___crtinit1__      DATA           DGROUP         0002:00003cdc   00000000
SET3___crtinit1__      DATA           DGROUP         0002:00003cdc   00000004
SET1___crtexit1__      DATA           DGROUP         0002:00003ce0   00000004
SET2___crtexit1__      DATA           DGROUP         0002:00003ce4   00000000
SET3___crtexit1__      DATA           DGROUP         0002:00003ce4   00000004
SET1___eh_frame__      DATA           DGROUP         0002:00003ce8   00000004
SET2___eh_frame__      DATA           DGROUP         0002:00003cec   00000008
SET3___eh_frame__      DATA           DGROUP         0002:00003cf4   00000004
SET1___eh_init__       DATA           DGROUP         0002:00003cf8   00000004
SET2___eh_init__       DATA           DGROUP         0002:00003cfc   00000004
SET3___eh_init__       DATA           DGROUP         0002:00003d00   00000004
SET1___eh_term__       DATA           DGROUP         0002:00003d04   00000004
SET2___eh_term__       DATA           DGROUP         0002:00003d08   00000004
SET3___eh_term__       DATA           DGROUP         0002:00003d0c   00000004
SET1___fork_parent1__  DATA           DGROUP         0002:00003d10   00000004
SET2___fork_parent1__  DATA           DGROUP         0002:00003d14   00000000
SET3___fork_parent1__  DATA           DGROUP         0002:00003d14   00000004
SET1___fork_child1__   DATA           DGROUP         0002:00003d18   00000004
SET2___fork_child1__   DATA           DGROUP         0002:00003d1c   00000000
SET3___fork_child1__   DATA           DGROUP         0002:00003d1c   00000004
________DATA           DATA           DGROUP         0002:00003d20   00000000
BSS32                  BSS            DGROUP         0002:00003d20   00000160
c_common               BSS            DGROUP         0002:00003e80   00000000
________BSS            BSS            DGROUP         0002:00003e80   00000000


                        +----------------+
                        |   Memory Map   |
                        +----------------+

* = unreferenced symbol
+ = symbol only referenced locally

Address        Symbol
=======        ======

Module: U:\usr\lib\dll0hi.obj({standard input})
0001:00000000* __text
0002:00000000* __data
0002:00000000* ___data_start
0002:00003d20* ___bss_start
0002:00003cc0+ __os2dll
0002:00003cc8  ___CTOR_LIST__
0002:00003cd0  ___DTOR_LIST__
0002:00003cd8* ___crtinit1__
0002:00003ce0* ___crtexit1__
0002:00003ce8  ___eh_frame__
0002:00003cf8  ___eh_init__
0002:00003d04  ___eh_term__
0002:00003d10+ ___fork_parent1__
0002:00003d18+ ___fork_child1__
Module: U:/tmp\ldconv_socketmodule_obj_19ea52885a3a128c58.obj(U:\DEV\python-2.7.5\Modules\socketmodule.c)
0001:00001f43* _fake_gai_strerror
0001:00001f5c* _fake_freeaddrinfo
0001:00001f9e* _fake_getaddrinfo
0001:0000379a* _fake_getnameinfo
0001:00005614+ _init_sockobject
0001:000065d3  _init_socket
Module: U:/tmp\ldconv_timemodule_obj_19ea52885a3a12e248.obj(U:\DEV\python-2.7.5\Modules\timemodule.c)
0001:000084f1* __PyTime_DoubleToTimet
0001:00008593+ _inittime
0001:0000871e  __PyTime_FloatTime
Module: U:\usr\local473\lib\libc_dll.lib(dllinit.obj)
0001:00008ad0  _DLL_InitTerm
Module: U:\usr\lib\libend.lib(src/libend/386/endlink386.asm)
0002:00003e80  _end
0002:00003d20  _edata
Module: U:\usr\lib\libend.lib(src/libend/386/end.asm)
0001:000096b0* _etext
0001:000096b0* __etext
0000:00000000* WEAK$ZERO
0002:00003e80  __end
0002:00003d20  __edata
Module: U:\usr\local473\lib\libc_dll.lib(setsockopt.obj)
0001:00008b30  _setsockopt
Module: U:\usr\local473\lib\libc_dll.lib(getsockopt.obj)
0001:00008c30  _getsockopt
Module: U:\usr\local473\lib\libc_dll.lib(shutdown.obj)
0001:00008d10  _shutdown
Module: U:\usr\local473\lib\libc_dll.lib(listen.obj)
0001:00008db0  _listen
Module: U:\usr\local473\lib\libc_dll.lib(connect.obj)
0001:00008e50  _connect
Module: U:\usr\local473\lib\libc_dll.lib(send.obj)
0001:00008ef0  _send
Module: U:\usr\local473\lib\libc_dll.lib(recv.obj)
0001:00008fa0  _recv
Module: U:\usr\local473\lib\libc_dll.lib(sendto.obj)
0001:00009050  _sendto
Module: U:\usr\local473\lib\libc_dll.lib(bind.obj)
0001:00009100  _bind
Module: U:\usr\local473\lib\libc_dll.lib(recvfrom.obj)
0001:000091a0  _recvfrom
Module: U:\usr\local473\lib\libc_dll.lib(getpeername.obj)
0001:00009270  _getpeername
Module: U:\usr\local473\lib\libc_dll.lib(getsockname.obj)
0001:00009310  _getsockname
Module: U:\usr\local473\lib\libc_dll.lib(accept.obj)
0001:000093b0  _accept
Module: U:\usr\local473\lib\libc_dll.lib(socket.obj)
0001:00009490  _socket
Module: U:\usr\local473\lib\libc_dll.lib(socketpair.obj)
0001:00009510  _socketpair
Module: U:\tmp\ldconv_libgcc_so_d_a_19ea52885a3b1abe0.lib(emx-ctordtor.obj)
0001:000095d0  ___ctordtorInit
0001:00009604  ___ctordtorTerm
Module: U:\tmp\ldconv_libgcc_so_d_a_19ea52885a3b1abe0.lib(emx-eh.obj)
0001:00009640  ___ehInit
0001:00009676* ___ehTerm


                        +----------------------+
                        |   Imported Symbols   |
                        +----------------------+

Symbol                              Module
======                              ======

___libc_ForkRegisterModule          libc065
___init_dll                         libc065
___libc_Back_termDll                libc065
___libc_ForkDeregisterModule        libc065
__atfork_callback                   libc065
_PyArg_ParseTuple                   python27
__Py_NoneStruct                     python27
_PyErr_Clear                        python27
_PyInt_FromLong                     python27
_PyErr_SetFromErrno                 python27
_PyEval_SaveThread                  python27
_PyEval_RestoreThread               python27
_PyFile_FromFile                    python27
_PyFile_SetBufSize                  python27
_PyString_FromStringAndSize         python27
__PyString_Resize                   python27
_PyErr_SetString                    python27
_PyOS_snprintf                      python27
_PyString_FromString                python27
_inet_ntop                          tcpip32
_PyExc_ValueError                   python27
_PyErr_Format                       python27
_inet_pton                          tcpip32
_PyLong_FromUnsignedLong            python27
_PyLong_AsUnsignedLong              python27
_PyErr_Occurred                     python27
_PyExc_TypeError                    python27
_PyExc_OverflowError                python27
__PyInt_AsInt                       python27
_PyFloat_FromDouble                 python27
_PyFloat_AsDouble                   python27
_inet_ntoa                          tcpip32
_inet_aton                          tcpip32
_getprotobyname                     tcpip32
_getservbyport                      tcpip32
_getservbyname                      tcpip32
__errno                             libc065
_gethostname                        tcpip32
_PyBuffer_Release                   python27
_PyErr_CheckSignals                 python27
_PyArg_ParseTupleAndKeywords        python27
_PyInt_FromSsize_t                  python27
_PyInt_AsLong                       python27
___libc_GLocaleCtype                libc065
___stderrp                          libc065
_gethostbyname                      tcpip32
_tcp_h_errno1                       tcpip32
_gethostbyaddr                      tcpip32
_PyThread_acquire_lock              python27
_PyThread_release_lock              python27
_Py_BuildValue                      python27
_PyErr_SetObject                    python27
_PyMem_Free                         python27
_PyArg_Parse                        python27
_PyTuple_Size                       python27
_PyList_New                         python27
_PyList_Append                      python27
_hstrerror                          tcpip32
_PyString_AsString                  python27
_PyLong_AsLong                      python27
_PyObject_CallMethod                python27
_PyTuple_Pack                       python27
_PyType_GenericNew                  python27
_PyType_Type                        python27
_Py_InitModule4                     python27
_PyExc_IOError                      python27
_PyErr_NewException                 python27
_PyModule_AddObject                 python27
__Py_ZeroStruct                     python27
_PyCapsule_New                      python27
_PyModule_AddIntConstant            python27
_PyThread_allocate_lock             python27
_PyObject_GenericGetAttr            python27
_PyType_GenericAlloc                python27
_PyObject_Free                      python27
_PyImport_ImportModuleNoBlock       python27
_PyDict_GetItemString               python27
_PyErr_NoMemory                     python27
_PyArg_UnpackTuple                  python27
_PyStructSequence_New               python27
DosSleep                            doscalls
_Py_IgnoreEnvironmentFlag           python27
_PyModule_GetDict                   python27
_PyStructSequence_InitType          python27
__CRT_init                          libc065
__CRT_term                          libc065
___libc_FH                          libc065
__libsocket_set_errno               tcpip32
__libsocket_setsockopt              tcpip32
__libsocket_sock_errno              tcpip32
__std_close                         libc065
__std_dup                           libc065
__std_fdopen                        libc065
__std_fclose                        libc065
__libsocket_getsockopt              tcpip32
__libsocket_shutdown                tcpip32
__libsocket_listen                  tcpip32
__std_select                        libc065
__libsocket_connect                 tcpip32
__libsocket_send                    tcpip32
__libsocket_recv                    tcpip32
__std_fcntl                         libc065
__std_free                          libc065
__std_fwrite                        libc065
__std_malloc                        libc065
__std_memset                        libc065
__std_memcpy                        libc065
__std_atoi                          libc065
__std_strcpy                        libc065
__std_sscanf                        libc065
__libsocket_sendto                  tcpip32
__libsocket_bind                    tcpip32
__std_sprintf                       libc065
__std_strchr                        libc065
__std_strerror                      libc065
__libsocket_recvfrom                tcpip32
__libsocket_getpeername             tcpip32
__libsocket_getsockname             tcpip32
__libsocket_accept                  tcpip32
___libc_TcpipAllocFH44              libc065
__libsocket_soclose                 tcpip32
__libsocket_socket                  tcpip32
__libsocket_socketpair              tcpip32
___libc_FHClose                     libc065
__std_strftime                      libc065
__std_time                          libc065
__std_localtime                     libc065
__std_asctime                       libc065
__std_clock                         libc065
__std_mktime                        libc065
__std_gettimeofday                  libc065
__std_ftime                         libc065
__std_ctime                         libc065
__std_gmtime                        libc065
__std_tzset                         libc065
__std_timezone                      libc065
__std_daylight                      libc065
__std_tzname                        libc065
__std_getenv                        libc065
___ctordtorInit1                    libc065
___ctordtorTerm1                    libc065
___register_frame_table             gcc473
___deregister_frame                 gcc473


                        +--------------------+
                        |   Libraries Used   |
                        +--------------------+

U:\tmp\ldconv_python2_7_dll_a_19ea52885a3a132c80.lib
U:\tmp\ldconv_libgcc_so_d_a_19ea52885a3b1abe0.lib
U:\usr\lib\libc_alias.lib
U:\usr\local473\lib\libc_dll.lib
U:\usr\lib\libos2.lib
U:\usr\lib\libend.lib


                        +-----------------------+
                        |   Linker Statistics   |
                        +-----------------------+

Stack size:  0000 (0.)
Memory size:  d530 (54576.)
Link time: 00:00.06
